:020000040000FA
:100000000AEF03F0F76A140FF66E000EF7220900EC
:10001000F550120053746570706572204D6F746FE7
:100020007220496E746572666163652076312C209A
:1000300062726F7567687420746F20796F752062C3
:10004000793A0A0D0000F76A560FF66E000EF72295
:100050000900F5501200416E647265772057696C93
:10006000736F6E0A0D00F76A760FF66E000EF722B8
:100070000900F55012007265636F6E6E73776F72D0
:100080006C642E636F6D0A0D00008E0E006E14C03E
:1000900001F013C002F0036A015209E102C001F04D
:1000A000026A080E005E015202E1006A08D0D89090
:1000B00001BE04D0023601360006F9D7019E0000C9
:1000C00090EF03F01750D8B471D0006E1B50D8B425
:1000D0006DD0002604E3810E002668E204D07F0E76
:1000E000005E64E363E018C01FF01C501F1A188EF6
:1000F0001C8E1A501E02F4CF21F019501D02F4CFAD
:1001000003F0F3CF20F01E02F3502126F4502022FA
:10011000000E03221A501D02F3502126F450202213
:10012000000E026A0322022218501E02F3502026FB
:10013000F4500322000E022218501D02F350032631
:10014000F4500222000E016A01221A501C02F350E0
:100150002026F4500322000E0222012219501C0214
:10016000F3500326F4500222000E012218501C0204
:10017000F3500226F4500122002A01BE05D0203699
:100180000336023601360006000E20AE0AD0032ADE
:1001900002220122015005E1025003E1035001E176
:1001A000002A1FBE018E1FAE019E04D0006A016AA4
:1001B000026A036A0000000C1750D8B4A6D0236E60
:1001C0001B50D8B4A2D0235E01E205D07F0E2326B7
:1001D000D8B09BD006D0810E235ED8A096D0D8B4DC
:1001E00094D023C000F0016A026A036A226A18C030
:1001F00021F0218E19C020F01AC01FF0190E236EB5
:100200001E501F5E0DE2010E205E0AE2215E08E232
:10021000225E06E2222A212A202A1E501F2628D0EA
:100220001D50205E12E2010E215E0FE2225E0DE201
:10023000222A212A1D5020261E501F2619E3202A7B
:1002400017E1212A15E1222A13D01C508009215ED2
:100250000EE2010E225E0BE2222A1C5080092126AA
:100260001D502026E9E3212AE7E1222AE5D7038071
:10027000232E01D00BD0D8901F36203621362236BF
:10028000D8900336023601362436BAD724A006D0D9
:10029000D890013202320332243202D0000635E017
:1002A00024BE1ED0D8901F362036213622361E504E
:1002B0001F5E07E2010E205E04E2215E02E2225E82
:1002C0001AE31D50205E05E2010E215E02E2225E6D
:1002D00012E31C508009215E03E2010E225E0BE353
:1002E000032A09E1022A07E1012A05E1002A0DE0BB
:1002F00001320232033218C023F01C50231A23AEFD
:1003000002D0018E06D0019E04D0006A016A026A02
:10031000036A0000B5EF03F0800ED8B2201A256AF8
:10032000266A1CC024F02050241A1B50D8B4DED0FA
:10033000236E23C000F01F50D8B4E1D0235ED8B4A0
:1003400082D001E23DD020C029F0298E21C028F0C2
:1003500022C027F0266AD890293228322732263246
:10036000232EF8D724AE03D02580DDD0259023900E
:100370002588EA6A1E0EE96EE9D0259824BE0AD0C7
:1003800023A013D02932283227322632002AD8B4AB
:10039000C5D00BD029BE0CD0D890263627362836AB
:1003A00029360006D8B4BAD0F5D7258C6BD0259C59
:1003B0001CC024F01CAE02D0298EA9D0299EA7D043
:1003C0001FC023F01FC000F01B50235E1CC029F08B
:1003D000298E1DC028F01EC027F0266AD890293229
:1003E000283227322632232EF8D724AE03D0258296
:1003F0009AD025922390258AEA6A220EE96EA6D029
:10040000259A24BE0AD023A013D0293228322732BD
:100410002632002AD8B482D00BD029BE0CD0D89076
:1004200026362736283629360006D8B477D0F5D7B1
:10043000258E28D0259E20C024F020AE02D0298E03
:1004400066D0299E64D020C029F0298E21C028F0D2
:1004500022C027F024AE04D0299E258464D02594A0
:10046000266A2390EA6A1E0EE96E70D024BE1CD064
:100470001CC024F023A006D029322832273226328D
:10048000002A4CE026AE0BD0272A09E1282A07E1F2
:10049000292A05E1293228322732002A3FE025BCEB
:1004A00086D725BEC7D71CD0800E291A29AE04D006
:1004B0003AD020C024F00AD01CC024F0295206E112
:1004C000285204E1275202E1006A21D029BE08D057
:1004D000D8902636273628362936002EF7D71ED054
:1004E00024AE02D0298E13D0299E11D01FC000F057
:1004F00020C029F021C028F022C027F008D01BC05E
:1005000000F01CC029F01DC028F01EC027F029C033
:1005100001F028C002F027C003F034D0006A016A5D
:10052000026A036A2FD0266A271E281E291E261E4D
:10053000262A05E1272A03E1282A01E1292A25B0F4
:1005400015D725B256D725B48AD7B3D7EF5027266B
:1005500005E3282A03E1292AD8B42380ED52EF507D
:10056000282603E3292AD8B42380ED52EF50EFBEAA
:1005700001D0800A2926D8B0238025B8FED625BA16
:100580003FD774D70000DCEF03F08E0E006E1B50D7
:10059000005E1CC002F01DC001F0028E005209E096
:1005A000D890025202E1015204E002320132002EE0
:1005B000F7D71CAE05D0011E021E012AD8B4022AAC
:1005C0000000E5EF03F0CE50CFCF03F0056E03C07F
:1005D00006F0CF6A090ECE6E0650085C09E303E10F
:1005E0000750055C05E20550075E0650085A02D028
:1005F000086A076A06500E5C09E303E10D50055CCA
:1006000005E205500D5E06500E5A02D00E6A0D6AC4
:10061000F4EF03F0F86AD09EEA6AE96AC150C00BB1
:100620000309C16E070EB46EB450A19CB896810E3A
:10063000AF6E260EAC6E900EAB6E056A066A076A48
:10064000086A096A0A6A0B6A0C6A0D6A0E6A850EE4
:10065000CD6E136A1350D6DC132A006E00509EA88C
:10066000FED7AD6E300E135CF5E1136A1350EBDC70
:10067000132A006E00509EA8FED7AD6E0F0E135CBD
:10068000F5E1136A1350EFDC132A006E00509EA8A8
:10069000FED7AD6E120E135CF5E1C150C00B0D0913
:1006A000C16EC050C00B0709C06EC09EC280040E50
:1006B000016EC250C30B0110C26E0A6A8C0E096E25
:1006C000130E0C6E880E0B6E93908A9093948A840E
:1006D000126A116A0D5208E10E5206E19290897079
:1006E0000CC00EF00BC00DF01150A008D8A471D0B2
:1006F000125086086EE1126A116AC282C2B2FED737
:10070000C450106A0F6E0F5206E1105204E10A6ADB
:10071000800E096E5ED010C014F00FC013F0B5D477
:100720001A6A196A186A7F0E176E03C01EF002C09B
:100730001DF001C01CF000C01BF0C4DC00C013F0B1
:1007400001C014F002C015F003C016F003C01AF087
:1007500002C019F001C018F000C017F01E6A1D6A2F
:100760007F0E1C6E860E1B6E27D51A6A200E196E20
:100770006D0E186E8B0E176E03C01EF002C01DF0BA
:1007800001C01CF000C01BF09DDC00C017F001C0D0
:1007900018F002C019F003C01AF0D89203C01EF07E
:1007A00002C01DF001C01CF000C01BF0226A216ACB
:1007B000206A860E1F6EB0D503C01EF002C01DF069
:1007C00001C01CF000C01BF0E0D602C00AF001C05E
:1007D00009F0075208E1085206E193928A720AC0B2
:1007E00008F009C007F0EFD6112AD8B4122A72D740
:0607F000010E016E030082
:020000040030CA
:0E00000000C20F1E008781000FC00FE00F40EE
:00000001FF
